:020000040800F2
:10000000E80800200101000865380008A93600084A
:10001000613800080D190008753A0008000000005A
:10002000000000000000000000000000513900083E
:1000300075190008000000006938000855390008EB
:100040001B0100081B0100081B0100081B01000820
:100050001B0100081B0100081B0100081B01000810
:100060001B0100081B0100081B0100081B01000800
:100070001B0100081B0100081B0100081B010008F0
:100080001B0100081B0100081B0100081B010008E0
:100090001B0100081B0100081B0100081B010008D0
:1000A0001B0100081B0100081B0100081B010008C0
:1000B0001B0100081B0100081B0100081B010008B0
:1000C0001B0100081B0100081B0100081B010008A0
:1000D0001B010008693A00081B0100081B01000809
:1000E0001B0100081B0100081B010008DFF80CD0F1
:1000F00000F018F800480047793A0008E8080020A6
:100100000648804706480047FEE7FEE7FEE7FEE7B1
:10011000FEE7FEE7FEE7FEE7FEE7FEE759390008E7
:10012000ED000008064C074D06E0E06840F00103D2
:1001300094E8070098471034AC42F6D3FFF7DAFF93
:10014000E4590008045A000840F210000021C2F2ED
:10015000000000228318815402F58072B2F5806F8E
:1001600019721974197683F8201083F8281083F80F
:10017000301083F8381083F8401083F8481083F863
:10018000501083F8581083F8601083F8681083F8D3
:10019000701083F8781083F8801083F8881083F843
:1001A000901083F8981083F8A01083F8A81083F8B3
:1001B000B01083F8B81083F8C01083F8C81083F823
:1001C000D01083F8D81083F8E01083F8E81083F893
:1001D000F01083F8F810BDD100210022831802F539
:1001E0008072B2F5806F597059725974597683F8DC
:1001F000211083F8291083F8311083F8391083F81F
:10020000411083F8491083F8511083F8591083F88E
:10021000611083F8691083F8711083F8791083F8FE
:10022000811083F8891083F8911083F8991083F86E
:10023000A11083F8A91083F8B11083F8B91083F8DE
:10024000C11083F8C91083F8D11083F8D91083F84E
:10025000E11083F8E91083F8F11083F8F910BDD1AB
:1002600000210022831802F58072B2F5806F997028
:1002700099729974997683F8221083F82A1083F87A
:10028000321083F83A1083F8421083F84A1083F84A
:10029000521083F85A1083F8621083F86A1083F8BA
:1002A000721083F87A1083F8821083F88A1083F82A
:1002B000921083F89A1083F8A21083F8AA1083F89A
:1002C000B21083F8BA1083F8C21083F8CA1083F80A
:1002D000D21083F8DA1083F8E21083F8EA1083F87A
:1002E000F21083F8FA10BDD100210022831802F524
:1002F0008072B2F5806FD970D972D974D97683F8CB
:10030000231083F82B1083F8331083F83B1083F805
:10031000431083F84B1083F8531083F85B1083F875
:10032000631083F86B1083F8731083F87B1083F8E5
:10033000831083F88B1083F8931083F89B1083F855
:10034000A31083F8AB1083F8B31083F8BB1083F8C5
:10035000C31083F8CB1083F8D31083F8DB1083F835
:10036000E31083F8EB1083F8F31083F8FB10BDD192
:1003700000210022831802F58072B2F5806F197196
:1003800019731975197783F8241083F82C1083F8E2
:10039000341083F83C1083F8441083F84C1083F831
:1003A000541083F85C1083F8641083F86C1083F8A1
:1003B000741083F87C1083F8841083F88C1083F811
:1003C000941083F89C1083F8A41083F8AC1083F881
:1003D000B41083F8BC1083F8C41083F8CC1083F8F1
:1003E000D41083F8DC1083F8E41083F8EC1083F861
:1003F000F41083F8FC10BDD100210022831802F50F
:100400008072B2F5806F597159735975597783F8B5
:10041000251083F82D1083F8351083F83D1083F8EC
:10042000451083F84D1083F8551083F85D1083F85C
:10043000651083F86D1083F8751083F87D1083F8CC
:10044000851083F88D1083F8951083F89D1083F83C
:10045000A51083F8AD1083F8B51083F8BD1083F8AC
:10046000C51083F8CD1083F8D51083F8DD1083F81C
:10047000E51083F8ED1083F8F51083F8FD10BDD179
:1004800000210022831802F58072B2F5806F997105
:1004900099739975997783F8261083F82E1083F84D
:1004A000361083F83E1083F8461083F84E1083F818
:1004B000561083F85E1083F8661083F86E1083F888
:1004C000761083F87E1083F8861083F88E1083F8F8
:1004D000961083F89E1083F8A61083F8AE1083F868
:1004E000B61083F8BE1083F8C61083F8CE1083F8D8
:1004F000D61083F8DE1083F8E61083F8EE1083F848
:10050000F61083F8FE10BDD100210022831802F5F9
:100510008072B2F5806FD971D973D975D97783F8A4
:10052000271083F82F1083F8371083F83F1083F8D3
:10053000471083F84F1083F8571083F85F1083F843
:10054000671083F86F1083F8771083F87F1083F8B3
:10055000871083F88F1083F8971083F89F1083F823
:10056000A71083F8AF1083F8B71083F8BF1083F893
:10057000C71083F8CF1083F8D71083F8DF1083F803
:10058000E71083F8EF1083F8F71083F8FF10BDD160
:1005900000F002BD2DE9F04F02FB02FCBCEB4C0F5A
:1005A00088BFBDE8F08F40F210084FF0000B4FF00D
:1005B000010EC2F2000800BF0BEB00058E1AF7B265
:1005C000EDB2FF0808EBC50506F00706EC5D0EFA74
:1005D00006F944EA0904EC55A0EB0B04E4B208EB7D
:1005E000C404E65D46EA0906E6555618F7B2FF0868
:1005F00006F0070914F807A00EFA09F64AEA0603FE
:10060000E355EB5D0BEB01043343EB551318E5B2F7
:10061000DBB2ED0808EBC30304F007045E5D0EFADD
:1006200004F946EA09065E55A1EB0B06F7B2FF088E
:1006300006F00706DC5D0EFA06F63443DC55831A35
:10064000DBB208EBC303DC5D3443DC550BF1010680
:1006500002FB02F706FB06775C5D67458CBF013A3B
:10066000B34602FB02F644EA0904BCEB460F5C55B4
:10067000A2DDBDE8F08F00002DE9F04F82B0151A21
:10068000B2EB000A18BF4FF0FF3A002D019544BFAE
:100690006A420192012DA3EB01044FF00102A8BFB1
:1006A00092465B1A9946019A1CBFC2F100094FF0AD
:1006B000FF33002CC4BFA1460123CB4600934A451B
:1006C000C8BF934600270022002400BF40F2100656
:1006D0005FFA80FEC2F20006C1F3C40806EBCE0E3C
:1006E00001F007031EF80860012505FA03F3DDF8A1
:1006F0002CC046EA0305BCF1000F08BF26EA03053B
:10070000019B07EB09061344B3EB0B02D4BF1A4657
:100710005044B6EB0B07D8BF3746009B04F10104E9
:10072000C8BF1944A3B29B450EF80850CED202B000
:10073000BDE8F08FB0B5CD0801F0070E40F2100112
:10074000C2F2000101EBC0004FF0010C415D0CFA58
:100750000EF341EA0304002A08BF21EA03044455CA
:10076000B0BD00002DE9F04182B040F60044C4F273
:10077000010420464FF480410022002601F0E4FDF0
:1007800020464FF48041012201F0DEFDAE208DF8BD
:10079000070020464FF48051002201F0D5FD40F2C1
:1007A0004045C2F200050DF10701284601224FF431
:1007B0007A7302F0F5FA4FF0200820464FF480518A
:1007C00000228DF8078001F0BFFD0DF107012846DA
:1007D00001224FF47A7302F0E3FA102720464FF417
:1007E000805100228DF8077001F0AEFD0DF1070178
:1007F000284601224FF47A7302F0D2FAB0208DF825
:10080000070020464FF48051002201F09DFD0DF1BC
:100810000701284601224FF47A7302F0C1FAC8207A
:100820008DF8070020464FF48051002201F08CFD26
:100830000DF10701284601224FF47A7302F0B0FA55
:1008400020464FF4805100228DF8076001F07CFDB6
:100850000DF10701284601224FF47A7302F0A0FA45
:1008600020464FF4805100228DF8077001F06CFD96
:100870000DF10701284601224FF47A7302F090FA35
:1008800040208DF8070020464FF48051002201F0EF
:100890005BFD0DF10701284601224FF47A7302F047
:1008A0007FFA81208DF8070020464FF48051002206
:1008B00001F04AFD0DF10701284601224FF47A7339
:1008C00002F06EFAFF208DF8070020464FF48051A9
:1008D000002201F039FD0DF10701284601224FF4F5
:1008E0007A7302F05DFAA1208DF8070020464FF4DC
:1008F0008051002201F028FD0DF107012846012258
:100900004FF47A7302F04CFAA6208DF807002046C7
:100910004FF48051002201F017FD0DF10701284628
:1009200001224FF47A7302F03BFAA8208DF80700F9
:1009300020464FF48051002201F006FD0DF1070121
:10094000284601224FF47A7302F02AFA3F208DF8EC
:10095000070020464FF48051002201F0F5FC0DF114
:100960000701284601224FF47A7302F019FAA420F5
:100970008DF8070020464FF48051002201F0E4FC7E
:100980000DF10701284601224FF47A7302F008FAAC
:10099000D3208DF8070020464FF48051002201F04B
:1009A000D3FC0DF10701284601224FF47A7302F0BF
:1009B000F7F920464FF4805100228DF8076001F0CE
:1009C000C3FC0DF10701284601224FF47A7302F0AF
:1009D000E7F9D5208DF8070020464FF4805100221A
:1009E00001F0B2FC0DF10701284601224FF47A73A1
:1009F00002F0D6F9F0208DF8070020464FF4805120
:100A0000002201F0A1FC0DF10701284601224FF45C
:100A10007A7302F0C5F9D9208DF8070020464FF40B
:100A20008051002201F090FC0DF1070128460122BF
:100A30004FF47A7302F0B4F922208DF807002046B3
:100A40004FF48051002201F07FFC0DF10701284690
:100A500001224FF47A7302F0A3F9DA208DF807002F
:100A600020464FF48051002201F06EFC0DF1070189
:100A7000284601224FF47A7302F092F912208DF881
:100A8000070020464FF48051002201F05DFC0DF17B
:100A90000701284601224FF47A7302F081F9DB2026
:100AA0008DF8070020464FF48051002201F04CFCE5
:100AB0000DF10701284601224FF47A7302F070F914
:100AC00020464FF4805100228DF8078001F03CFC55
:100AD0000DF10701284601224FF47A7302F060F904
:100AE0008D208DF8070020464FF48051002201F040
:100AF0002BFC0DF10701284601224FF47A7302F016
:100B00004FF914208DF8070020464FF48051002241
:100B100001F01AFC0DF10701284601224FF47A7307
:100B200002F03EF9AF208DF8070020464FF48051C7
:100B3000002201F009FC0DF10701284601224FF4C3
:100B40007A7302F02DF940F21000C2F20000002189
:100B50004218465401F58071B1F5806F1672167413
:100B6000167682F8206082F8286082F8306082F879
:100B7000386082F8406082F8486082F8506082F8FD
:100B8000586082F8606082F8686082F8706082F86D
:100B9000786082F8806082F8886082F8906082F8DD
:100BA000986082F8A06082F8A86082F8B06082F84D
:100BB000B86082F8C06082F8C86082F8D06082F8BD
:100BC000D86082F8E06082F8E86082F8F06082F82D
:100BD000F860BDD100210022831802F58072B2F5C1
:100BE000806F597059725974597683F8211083F8BF
:100BF000291083F8311083F8391083F8411083F8F5
:100C0000491083F8511083F8591083F8611083F864
:100C1000691083F8711083F8791083F8811083F8D4
:100C2000891083F8911083F8991083F8A11083F844
:100C3000A91083F8B11083F8B91083F8C11083F8B4
:100C4000C91083F8D11083F8D91083F8E11083F824
:100C5000E91083F8F11083F8F910BDD100210022CA
:100C6000831802F58072B2F5806F99709972997449
:100C7000997683F8221083F82A1083F8321083F8CB
:100C80003A1083F8421083F84A1083F8521083F820
:100C90005A1083F8621083F86A1083F8721083F890
:100CA0007A1083F8821083F88A1083F8921083F800
:100CB0009A1083F8A21083F8AA1083F8B21083F870
:100CC000BA1083F8C21083F8CA1083F8D21083F8E0
:100CD000DA1083F8E21083F8EA1083F8F21083F850
:100CE000FA10BDD100210022831802F58072B2F5FE
:100CF000806FD970D972D974D97683F8231083F8AC
:100D00002B1083F8331083F83B1083F8431083F8DB
:100D10004B1083F8531083F85B1083F8631083F84B
:100D20006B1083F8731083F87B1083F8831083F8BB
:100D30008B1083F8931083F89B1083F8A31083F82B
:100D4000AB1083F8B31083F8BB1083F8C31083F89B
:100D5000CB1083F8D31083F8DB1083F8E31083F80B
:100D6000EB1083F8F31083F8FB10BDD100210022B3
:100D7000831802F58072B2F5806F197119731975B5
:100D8000197783F8241083F82C1083F8341083F833
:100D90003C1083F8441083F84C1083F8541083F807
:100DA0005C1083F8641083F86C1083F8741083F877
:100DB0007C1083F8841083F88C1083F8941083F8E7
:100DC0009C1083F8A41083F8AC1083F8B41083F857
:100DD000BC1083F8C41083F8CC1083F8D41083F8C7
:100DE000DC1083F8E41083F8EC1083F8F41083F837
:100DF000FC10BDD100210022831802F58072B2F5EB
:100E0000806F597159735975597783F8251083F894
:100E10002D1083F8351083F83D1083F8451083F8C2
:100E20004D1083F8551083F85D1083F8651083F832
:100E30006D1083F8751083F87D1083F8851083F8A2
:100E40008D1083F8951083F89D1083F8A51083F812
:100E5000AD1083F8B51083F8BD1083F8C51083F882
:100E6000CD1083F8D51083F8DD1083F8E51083F8F2
:100E7000ED1083F8F51083F8FD10BDD1002100229C
:100E8000831802F58072B2F5806F99719973997524
:100E9000997783F8261083F82E1083F8361083F89C
:100EA0003E1083F8461083F84E1083F8561083F8EE
:100EB0005E1083F8661083F86E1083F8761083F85E
:100EC0007E1083F8861083F88E1083F8961083F8CE
:100ED0009E1083F8A61083F8AE1083F8B61083F83E
:100EE000BE1083F8C61083F8CE1083F8D61083F8AE
:100EF000DE1083F8E61083F8EE1083F8F61083F81E
:100F0000FE10BDD100210022831802F58072B2F5D7
:100F1000806FD971D973D975D97783F8271083F881
:100F20002F1083F8371083F83F1083F8471083F8A9
:100F30004F1083F8571083F85F1083F8671083F819
:100F40006F1083F8771083F87F1083F8871083F889
:100F50008F1083F8971083F89F1083F8A71083F8F9
:100F6000AF1083F8B71083F8BF1083F8C71083F869
:100F7000CF1083F8D71083F8DF1083F8E71083F8D9
:100F8000EF1083F8F71083F8FF10BDD100F004F8DC
:100F900002B0BDE8F08100002DE9F04F81B040F6CD
:100FA000004440F2100640F24045C4F20104C2F28F
:100FB0000006C2F200050DF101090DF1020B0DF161
:100FC00003074FF0000800BFA8F150008DF80000A3
:100FD00020464FF48051002201F0B6F928466946B8
:100FE00001224FF47A7301F0DBFE00208DF801003E
:100FF00020464FF48051002201F0A6F928464946C8
:1010000001224FF47A7301F0CBFE10208DF802001C
:1010100020464FF48051002201F096F928465946A7
:1010200001224FF47A7301F0BBFE6FF0070A00BF94
:1010300006EB0A00007A4FF480518DF80300204639
:10104000012201F081F92846394601224FF47A73D2
:1010500001F0A6FE0AF1080ABAF57E7FE8D108F190
:101060000108B8F1080F06F10106ADD101B0BDE8E5
:10107000F08F00002DE9F04F87B0082B049001D1CC
:1010800006250BE0D80801275E0718BF07EBD30041
:101090005F087843C5B2002D00F02281A2F1200044
:1010A000C2B25808039043F6EA7002EB4207C0F65A
:1010B000000000EB470944F286600197C0F600008B
:1010C000049F4FF0000C00EB021002920090059379
:1010D00008E000BF069D0CF1010C013D09F101097A
:1010E00000F0FE80082B4E461ED0182B0CD0102B83
:1010F00016D00C2B40F0F480019A44F21220C0F676
:10110000000000EB820608E0029A44F6764002EB0B
:10111000C206C0F6000000EB8606664404E000BF8D
:10112000009800EB0C0600BF40F2100096F900B0EA
:10113000FEB2CAB2C2F20000D20800EBC60801F04B
:10114000070418F80260012000FA04F426EA040AF1
:10115000DDF840E0344356460695BEF1000F04BF6B
:10116000264654465FEACB7508BF344608F802406D
:101170004A1CD4B2E40802F0070218F8045000FA3E
:1011800002F225EA02062A433546BEF1000F04BFEB
:10119000154632465FEA8B7658BF2A4608F8042087
:1011A0008A1CD4B2E40802F0070218F8045000FACE
:1011B00002F225EA02062A433546BEF1000F04BFBB
:1011C000154632465FEA4B7658BF2A4608F8042097
:1011D000CA1CD4B2E40802F0070218F8045000FA5E
:1011E00002F225EA02062A433546BEF1000F04BF8B
:1011F000154632465FEA0B7658BF2A4608F80420A7
:101200000A1DD4B2E40802F0070218F8045000FAEC
:1012100002F225EA02062A433546BEF1000F04BF5A
:10122000154632465FEACB6658BF2A4608F80420C6
:101230004A1DD4B2E40802F0070218F8045000FA7C
:1012400002F225EA02062A433546BEF1000F04BF2A
:10125000154632465FEA8B6658BF2A4608F80420D6
:101260008A1DD4B2E40802F0070218F8045000FA0C
:1012700002F225EA02062A433546BEF1000F04BFFA
:10128000154632465FEA4B6658BF2A4608F80420E6
:10129000CA1DD4B2E40802F0070218F8045000FA9C
:1012A00002F225EA02062A4335463B46BEF1000F0C
:1012B00004BF15463246BBF1000F58BF2A46059BB6
:1012C0000137082B08F804203FF404AF049CFAB25D
:1012D000039E121BB24204BF27460831FAE600BF44
:1012E00007B0BDE8F08F00002DE9F04F85B0019206
:1012F000DA0801275E0718BF07EBD30202FB03FCE5
:10130000BCF1000F0493039000F012810498103890
:10131000C2B2400140EAD200C3B2062B00F20881FB
:101320004FF0010E0EFA03F010F0470F00F00081AD
:1013300043F6C230019AC0F6000000EB421943F6B2
:101340006A50C0F6000000EBC2100E9D009003989A
:1013500000270293D2E000BF009AD61940F2100392
:1013600096F900A0C6B2CAB2C2F20003D20803EBDB
:10137000C60801F0070B18F802600EFA0BF326EA14
:10138000030433432646002D04BF1E4623465FEA6E
:10139000CA7408BF334608F802304A1CD3B2DB08CF
:1013A00002F0070218F803400EFA02F224EA0206DD
:1013B00022433446002D04BF144632465FEA8A7643
:1013C00058BF224608F803208A1CD3B2DB0802F07B
:1013D000070218F803400EFA02F224EA020622433A
:1013E0003446002D04BF144632465FEA4A7658BFA1
:1013F000224608F80320CA1CD3B2DB0802F0070219
:1014000018F803400EFA02F224EA02062243344698
:10141000002D04BF144632465FEA0A7658BF2246C2
:1014200008F803200A1DD3B2DB0802F0070218F8FF
:1014300003400EFA02F224EA020622433446002D4B
:1014400004BF144632465FEACA6658BF224608F80F
:1014500003204A1DD3B2DB0802F0070218F803404C
:101460000EFA02F224EA020622433446002D04BF9B
:10147000144632465FEA8A6658BF224608F80320BF
:101480008A1DD3B2DB0802F0070218F803400EFAF7
:1014900002F224EA020622433446002D04BF144619
:1014A00032465FEA4A6658BF224608F80320CA1D42
:1014B000D3B2DB0802F0070218F803400EFA02F27A
:1014C00024EA020622433446002D04BF1446324665
:1014D000BAF1000F58BF22460130039C08F80320E0
:1014E000C2B2049B121B9A4204BF08312046029BE1
:1014F0000137BCF1010C09F1010919D0022B3FF4AD
:101500002BAF012B08D0002B4E463FF427AF43F6FC
:10151000EA52C0F6000220E7019A02EBC20643F647
:101520002252C0F6000202EBC6063E4416E700BF98
:1015300005B0BDE8F08F00002DE9F04F85B0002B1D
:10154000049167D00E9982464D080220082908BFF1
:1015500000EB5105981E029058421C4616464FF06B
:1015600000095FFA80FB42F21078039223E000BF8B
:101570000120B6FBF0F04CF6CD41CCF6CC41A0FBFF
:101580000112D10801EB8101A0EB410009FB05A18B
:1015900040F03002002808BF3022C8B20499DDE9CB
:1015A0000E37D2B20097FFF765FD09F101095FFA26
:1015B00089F0A0422ED26FEA0900C1B25945D7D0B6
:1015C0000299A1EB0901C9B2032900EB040101D280
:1015D000012009E001F0FC02002301200433DEB207
:1015E000964200FB08F0F9D1039E11F00301C0D030
:1015F000012903D100EB80004000BAE74FF47A7272
:10160000424302294FF0640108BF00FB01F210467B
:10161000AFE700BF05B0BDE8F08F00002DE9F04F47
:1016200082B0DF085D0700924FF0010618BF06EB9D
:10163000D307002F00F0E18084460098002800F0D6
:10164000DC800B9C0098A4F1010A00FB07F36646BE
:101650004FF001090120012B98BF034640F2100210
:101660000193F7B2CBB2C2F2000260464FEAD30C4C
:1016700002EBC70701F0070417F80C5009FA04F44D
:10168000DDF830E01AF901BF25EA04082C43BEF169
:10169000000F454604BF254644465FEACB7301F17F
:1016A000010308BF2C46DDB207F80C40ED0803F03B
:1016B00007037C5D09FA03F3844624EA030023430D
:1016C000BEF1000F024604BF1A4603465FEA8B7064
:1016D00001F1020058BF1346C2B27B55D20800F098
:1016E0000700BB5C09FA00F023EA000518432B460B
:1016F000BEF1000F04BF034628465FEA4B7558BF92
:101700001846B854C81CC2B2D20800F00700BB5C2F
:1017100009FA00F023EA000518432B46BEF1000F3A
:1017200004BF034628465FEA0B7558BF1846B854F5
:10173000081DC2B2D20800F00700BB5C09FA00F035
:1017400023EA000518432B46BEF1000F04BF0346F1
:1017500028465FEACB6558BF1846B854481DC2B248
:10176000D20800F00700BB5C09FA00F023EA00058C
:1017700018432B46BEF1000F04BF034628465FEA1C
:101780008B6558BF1846B854881DC2B2D20800F005
:101790000700BB5C09FA00F023EA000518432B465A
:1017A000BEF1000F04BF034628465FEA4B6558BFF1
:1017B0001846B854C81DC2B2D20800F00700BB5C7E
:1017C00009FA00F023EA000518432B46BEF1000F8A
:1017D00004BF034628460136BBF1000F58BF184628
:1017E000F3B2009DA3EB0C03AB42019B04BF664622
:1017F0000831013BB8547FF431AF02B0BDE8F08F3F
:101800002DE9F04381B0994613780D46A3F12001EC
:10181000C9B25E291BD8DDF8208006464FEA590779
:10182000541EB9F1080F08BF062700BFF0B2DAB2A4
:1018300029464B46CDF80080FFF71CFCA3783E44B8
:10184000A3F12000C0B25F2804F10104EED301B07F
:10185000BDE8F083B0B582B0044600200190216855
:101860008A68D2074FD1886840F00100886040F252
:101870000800C2F2000000684DF68361C4F21B311B
:10188000A0FB0101880C01900198A0B101980138DA
:101890000190019878B1019801380190019850B1F8
:1018A000019801380190019828B101980138019000
:1018B00001980028EAD100F04DFD21688968C90728
:1018C0001CD1054603E000BF8068C0071AD100F0B4
:1018D00041FD411B20680329F6D38168C907F3D174
:1018E000A06A40F01000A062E06A40F00100E062EF
:1018F000002084F82400012002B0B0BD002002B016
:10190000B0BD00BF002002B0B0BD0000FEE7000087
:1019100070B540F69972C0F6000240F2491C0262AE
:1019200040F2357240F2796340F2955E41F6010172
:1019300041F2E92441F2395541F21D66C0F6000C2E
:10194000C0F60002C0F60003C0F6000EC0F60001AB
:10195000C0F60004C0F60005C0F60006C0E9001598
:10196000C0E90242C0E9043EC0E9066CFEF7FAFE97
:1019700070BD000070470000EFF3108072B600BF2A
:10198000FEE7000010B581B00022009290F82420FC
:10199000012A03D10221084601B010BD4B68012283
:1019A000062B80F8242017D8D0F800C003EB83035F
:1019B0005A1F1F23DCF834E003FA02F40B682EEA06
:1019C000040403FA02F22243CCF83420092B03EB7F
:1019D000430219D936E000BFD0F800C00C2B03EB4E
:1019E00083021DD8233A1F23DCF830E003FA02F407
:1019F0000B682EEA040403FA02F22243CCF83020EA
:101A0000092B03EB43021DD8DCF81030072489684A
:101A10009440A34391401943CCF81010002130E0CA
:101A2000413A1F23DCF82CE003FA02F40B682EEA9B
:101A3000040403FA02F22243CCF82C20092B03EB16
:101A40004302E1D9DCF80CE01E3A0724896894408F
:101A50002EEA0404914023F001022143102ACCF81D
:101A60000C100DD142F20841C4F20101A1F10802AB
:101A700094450DD0816A41F020018162012100E08E
:101A80000021002280F82420084601B010BD00BFCC
:101A90000A68120230D40A68102B42F400020A606D
:101AA0002CD140F20801C2F2000109684DF68362B0
:101AB000C4F21B32A1FB0212910C01EB810149001F
:101AC00000910099E1B10099013900910099C9B1E3
:101AD0000099013900910099B1B100990139009143
:101AE000009999B1009901390091009900294FF0AE
:101AF0000001E8D1C5E700BF0021C2E70021C0E72F
:101B00000021BEE70021BCE70021BAE70021B8E7C9
:101B10000068C06C70470000B0B5002800F0A880D5
:101B20000446806A20B121688868C0070BD114E0A0
:101B30000020E06284F82400204600F09BF8216831
:101B40008868C00709D0886820F00100886000F02C
:101B500001FC21688A68D20726D1A06AC0063AD45F
:101B6000A06A41F2021290430230A062E069D4E917
:101B7000013240EA030C531EB3FA83F35D091346A6
:101B8000B2F5807F18BF2B02207D257B01284CEA0F
:101B9000450030D135B3A56A45F02005A562E56A58
:101BA00045F00105E56226E0054602E08868C007C9
:101BB000D3D000F0CFFB401B21680328F6D3886800
:101BC000C007F3D0A06A40F01000A062E06A40F0C5
:101BD0000100E062A06AA06A40F01000A06201204B
:101BE000B0BD00BFD4F818C04EF60005CFF6FF75A3
:101BF00005EB4C352B434D68B2F5807F25F46945E4
:101C000043EA05034B608B684FF2FD75CFF6E17533
:101C100003EA050343EA00038B6001D0012A07D1E0
:101C200022690023CFF6F07303EB025201E000BFFC
:101C30000022CB6A23F470031A43CA62896840F613
:101C4000FE62CFF61F721140814207D10020E06290
:101C5000A16A012262F30101A162B0BDA06A40F055
:101C6000100020F00200A062E06A40F00100E06293
:101C70000120B0BD80B586B0014640F60040C4F2F8
:101C80000100096800F5C05291424FF00001CDE912
:101C9000041101D006B080BD41F21801C4F2020166
:101CA0000A6842F400720A600A6802F40072019243
:101CB000019A0A6842F008020A60096801F0080106
:101CC000019101990321CDE9021102A900F02EFA38
:101CD00006B080BDF0B581B000270D4604460097E0
:101CE00000F038FB21688A68D20543D4064648686C
:101CF000C00503D4C86A10F4700F45D040F2080044
:101D0000C2F200000768022000F0E2FB216844F6FE
:101D100024130A69B7FBF0F0C2F292431A4206D1CB
:101D2000CA6844F62413C0F292031A425ED00A69CC
:101D300042F29243C1F249231A4207D1CA6842F2E1
:101D40009243C0F249031A4200F0C0800A6949F286
:101D50004923C0F224031A424FF0FC0257D1CF6846
:101D60001F4208BF5422009B02FB00F7BB4253D323
:101D7000C3E000BFA06A40F02000A06284F8247095
:101D8000012001B0F0BD00BF0868800700F1B580F8
:101D9000681C00F0A880FDB90868800772D5086843
:101DA000800700F1AA80086880076BD50868800763
:101DB00000F1A3800868800764D50868800700F1F7
:101DC0009C80086880075DD508688007E4D594E0AA
:101DD0000868800700F1918000F0BCFA801B216840
:101DE000A842F5D908688007F2D44BE00A6942F2AC
:101DF0009243C1F249231A424FF0290207D1CB681E
:101E000042F29247C0F249073B4208BF1422009BAE
:101E100002FB00F7BB4270D2681C4FD055BB009844
:101E2000B8422FD30098013000900098B84264D295
:101E30000098B84226D30098013000900098B8422C
:101E40005BD20098B8421DD30098013000900098F2
:101E5000B84252D20098B84214D300980130009092
:101E60000098B842DBD348E0009801300090009819
:101E7000B84233D200F06EFA801BA842F4D9009821
:101E8000B842F1D2A06A40F00400A062002084F8B9
:101E90002400032001B0F0BD0098013000900098AC
:101EA000B8422AD20098013000900098B84224D25B
:101EB0000098013000900098B8421ED2009801307E
:101EC00000900098B842E7D317E000BF5422009B6F
:101ED00002FB00F7BB429FD30FE000BF21680CE07C
:101EE0000868800709D40868800706D40868800756
:101EF0005CBF08685FEA8070F2D56FF0120008607E
:101F0000A06A40F40070A062886800F46020B0F518
:101F1000602F01D1207B18B1002001B0F0BD00BFBF
:101F2000A06A20F48070A062A06AC004F4D4A06A01
:101F300040F00100A062002001B0F0BD10B50446E1
:101F400090F82400012804BF022010BD012084F86D
:101F500024002046FFF77EFC20B1002184F82410E5
:101F600010BD00BF42F2044C2068A16AC4F2010C0B
:101F700040F2013291430CF57F7201F5807190427D
:101F8000A16233D0A16A21F48011A16241684905A0
:101F900004D5A16A012363F30D31A162A16A002374
:101FA000C9044FF0000144BFE16A21F00601E1627B
:101FB0006FF0020184F824300160816801F460212F
:101FC000B1F5602F06D190420AD1DCF8001011F46F
:101FD000702F05D0816841F480118160002010BD10
:101FE000816841F4A0018160002010BDDCF8001080
:101FF00011F4702FC6D0A16A41F48011A162DCF8FF
:1020000000104905C5D4C9E7014690F8210002280F
:1020100016D10868D1E90FC3026822F00E020260EF
:10202000026822F001020260012000FA03F2CCF8FB
:10203000042081F821000020002281F82020704730
:10204000042088630120002281F8202070470000CE
:1020500080B590F82110022924D10268116821F07E
:102060000E0111602F211368C4F202018A4240F26E
:102070000401C4F2020123F00103136016DD3023D2
:10208000C4F202039A421DD04423C4F202039A42CE
:102090001CD05823C4F202039A421DD14FF480335E
:1020A00022E000BF04218163012080BD0823C4F227
:1020B00002039A420ED01C23C4F202039A420BD1AF
:1020C000102311E04FF480730EE000BF4FF48053F3
:1020D0000AE000BF012307E001F1680C4FF08073B4
:1020E000624508BF4FF480130B60012180F8211076
:1020F000426B002180F820100AB190470021084669
:1021000080BD0000B0B5044600F024F9054640F259
:102110000000C2F200000078611C18BF044400BF38
:1021200000F018F9401BA042FAD3B0BD2DE9F04FE2
:1021300082B00E68002E00F0038141F20042C4F22A
:102140000102042340F2004E904208BF03234FF6E1
:10215000FF7CC4F2010E009300240123C1F2100C95
:102160004FF0000A4FF0000949E000BF012704F0DA
:102170000C030F229A402BEA020207FA03F34FEAFC
:102180009A051A4346F82520D1F804B040F20C45D0
:102190005FEACB22DEF8082054BF22EA080242EAB6
:1021A0000802C4F20105CEF808202A685FEA8B23F2
:1021B00054BF22EA080242EA08022A605FEA8B332F
:1021C000DEF8042054BF22EA080242EA08025FEA6D
:1021D000CB33CEF80420DEF800204FF0010354BFCB
:1021E00022EA080242EA0802CEF800200E680AF14C
:1021F000010A36FA0AF204F1040400F0A18003FA9D
:102200000AF816EA080FF1D04E68664512DC122E65
:1022100056D8DFE806F0350B454955555555555507
:10222000555555555555554D510000BFD1F80C9099
:1022300046E000BF4FF6FF72C1F2210296420FDC6A
:102240000022C1F2110296421AD00022C1F21202FB
:10225000964215D00022C1F22102964210D02FE002
:102260000022C1F2220296420AD00022C1F23102BB
:10227000964205D00022C1F23202964220D100BF20
:102280008A684AB1012A14BFC0F81480C0F81080CF
:102290004FF0080914E000BF4FF0040910E000BF40
:1022A000CA6802F108090BE04FF0000908E000BF1E
:1022B000CA6802F1040903E0CA6802F10C0900BF10
:1022C00022460646BAF1080F24BF203A0436376882
:1022D0000F25954027EA050509FA02F22A433260E4
:1022E000CA79D2067FF582AF41F21803C4F2020325
:1022F0001A68AEF57E7642F001021A601A6802F0A2
:1023000001020192019A2AF0030256F802B040F647
:102310000002C4F20102904210D040F60042C4F222
:10232000010290423FF422AF41F20002C4F20102E6
:10233000009F904208BF022719E700BF002716E759
:1023400002B0BDE8F08F0000002A08BF0904016157
:102350007047000040F2E040C2F2000000687047A1
:1023600040F2000040F2E041C2F20000C2F200017F
:1023700000780A68104408607047000080B542F297
:102380000000C4F20200016841F010010160032066
:1023900000F08EF80F2000F005F800F027F800207C
:1023A00080BD000070B540F20006C2F2000640F2A7
:1023B00008013278C2F200014FF47A730968B3FB66
:1023C000F2F20446B1FBF2F1084600F0E7FD0F2CF3
:1023D0004FF0010508D838B94FF0FF3021460022F0
:1023E000002500F039F87460284670BD82B041F2D3
:1023F0001800C4F202000168022241F001010160EC
:10240000016801F0010101910199416841F0805199
:102410004160406800F08050009000980420C4F2B1
:102420000100016862F31A61016002B070470000A8
:10243000002848BF7047C1B200F01F00012202FA15
:1024400000F04EF20012CEF2000242EAD10121F079
:10245000030108607047000010B54EF60C5CCEF228
:10246000000CDCF80030C3F3022E8EF00704042CBD
:1024700028BF0424BEF103034FF0FF3E0EFA04F41C
:1024800038BF0023A14399400EFA03F39A43114346
:1024900000F00F0200F160430901043A03F56443C0
:1024A0006244002848BF02F10C03197010BD0000FF
:1024B0004EF60C51CEF200010A684FF6FF031A40A7
:1024C00060F30A2242F0806040F0FD7008607047BF
:1024D00080B5012818D0022836D0102832D141F218
:1024E0000401C4F202010A6851F8040CC00129D5A4
:1024F000C2F383402DA3185CD2033DD440F60012F2
:10250000C0F23D02504343E041F20400C4F2020035
:10251000C16940F202320A40B2F5817F04BF4FF434
:10252000004080BD01F44071B1F5407F1CD0B1F591
:10253000007F07D1006A49F64041800701EAE07058
:1025400080BD00BF002080BD00F0B4F941F204015D
:10255000C4F2020109680222C1F3813102EB410198
:10256000B0FBF1F080BD00BF50F8040C4FF22441E5
:10257000800301EAE07080BD0A6810A3C2F3404204
:102580009A5C41F20023C0F27A03B3FBF2F25043AB
:102590000968490248BF80BD4AF6AB214000CAF62F
:1025A000AA21A0FB0101480880BD00BF0203040569
:1025B000060708090A0B0C0D0E0F1010010200008F
:1025C0002DE9F04182B00446007841F21C06C007B4
:1025D000C4F202064AD0306810F0805808D1306842
:1025E00040F080503060306800F0805001900198D9
:1025F00047F20007C4F200073868C00512D43868F3
:1026000040F480703860FFF7A5FE05463868C005C5
:1026100008D4FFF79FFE401B6428F7D9032002B0BF
:10262000BDE8F081706810F4407012D0616801F468
:10263000407188420DD0706840F24042C4F242229C
:10264000012320F4407113600023C0071360716000
:102650002AD17068616820F440700843B8F1000F17
:10266000706003D1306820F08050306020688107AE
:1026700007D556F8181CA26821F44041114346F8CA
:10268000181CC00604D4002002B0BDE8F08100BFD1
:1026900056F8180CE16820F48000084346F8180C3E
:1026A000002002B0BDE8F081FFF754FE054641F27C
:1026B000883700BF70688007CBD4FFF74BFE401B04
:1026C000B8424FF00300F5D9EBE700002DE9F043E5
:1026D00081B0002800F0858042F20008C4F20208B0
:1026E0000446D8F800000D4600F0070088420CD2DE
:1026F000D8F8000020F007002843C8F80000D8F8F8
:10270000000000F00700A8426BD1206841F20409E4
:102710008107C4F2020917D5410705D5D9F8001081
:1027200041F4E061C9F80010010705D5D9F800109F
:1027300041F46051C9F80010D9F80010A26821F0E6
:10274000F0011143C9F80010C00741D1D8F80000CA
:1027500000F00700A8420CD9D8F8000020F00700CC
:102760002843C8F80000D8F8000000F00700A8428D
:1027700037D12068410707D5D9F80010E26821F465
:10278000E0611143C9F80010000708D5D9F800002E
:10279000216920F4605040EAC100C9F80000D9F86E
:1027A000002002F00C00082841F20020C0F27A005C
:1027B00050D145F6D213C2F38341C0F60003595CF1
:1027C000D2033BD440F60010C0F23D00484341E044
:1027D000606802280AD001282AD159F8041C89030C
:1027E00008D4012001B0BDE8F08300BF59F8041CF3
:1027F0008901F6D5D9F8001021F003010843C9F882
:102800000000FFF7A7FD064641F28837D9F800001F
:10281000616800F00C00B0EB810F97D0FFF79AFDD4
:10282000801BB842F2D9032001B0BDE8F08300BF9D
:1028300059F8041C8907D4D5DCE700BFD9F800207B
:1028400043F6C033C2F34042C0F600039A5C4843EB
:10285000B0FBF2F0D9F8001043F6A832C1F303112F
:10286000C0F60002515C40F2080220FA01F140F289
:102870000400C2F200000068C2F200021160FFF71B
:1028800091FD002001B0BDE8F083000040F2080097
:1028900041F20401C2F20000C4F2020100680968BA
:1028A00043F6B832C1F30221C0F60002515CC840C1
:1028B0007047000040F2080041F20401C2F200003B
:1028C000C4F202010068096843F6B832C1F3C221BC
:1028D000C0F60002515CC840704700002DE9F0418D
:1028E00082B0002868D00446007841F20006C00794
:1028F000C4F2020625D0706800F00C0004281BD03A
:10290000706800F00C00082802D17068C00313D46E
:102910006068002800F06881B0F5A02F00F07C818D
:10292000B0F5803F00F07C81306820F4803030606A
:10293000306820F4802076E13068800301D560683B
:10294000D0B32078800718D5706810F00C0F07D02E
:10295000706800F00C0008286ED17068C0036BD45A
:102960003068800702D52069012825D13068616967
:1029700020F0F80040EAC1003060207800071FD442
:102980002078400732D4E56995B1706800F00C00FA
:10299000082840F08F80012D0ED07068216A00F465
:1029A00080328A4208D1616A00F47010884203D1F3
:1029B000002002B0BDE8F081012002B0BDE8F08146
:1029C000A069002862D00020C4F242200121C0F892
:1029D0008014FFF7BFFC0546706A800700F18C8009
:1029E000FFF7B8FC401B0228F6D92AE1F06910F085
:1029F000805808D1F06940F08050F061F06900F033
:102A000080500090009847F20007C4F20007386831
:102A1000C00529D4386840F480703860FFF79AFC0C
:102A2000054600BF3868C0051ED4FFF793FC401B65
:102A30006428F7D905E100BF2069002840F20000B2
:102A4000C4F2422000F0828001210160FFF782FC85
:102A5000054600BF306880073FF588AFFFF77AFC76
:102A6000401B0228F6D9ECE0E068002800F08080E6
:102A7000052800F09780012800F09880306A20F047
:102A800001003062306A20F0040092E00020C4F2BD
:102A900042200021C0F88014FFF75CFC054600BF0F
:102AA000706A80077FF56CAFFFF754FC401B02286B
:102AB000F6D9C6E00027C4F2422700203866FFF7A7
:102AC00049FC022D05460BD13068800140F1BE80E3
:102AD000FFF740FC401B02284FF00300F4D968E7E1
:102AE000306880017FF564AFFFF734FC401B02289B
:102AF0004FF00300F4D95CE740F20800C2F2000096
:102B0000006844F6D351C1F26201A0FB0101480AFA
:102B1000019000BF00BF0198411E002801913FF4C1
:102B20002FAF00BF0198411E002801913FF428AF4C
:102B300000BF0198411E002801913FF421AF00BF62
:102B40000198411E00280191E4D119E7002101609C
:102B5000FFF700FC054600BF306880077FF50DAF2A
:102B6000FFF7F8FB401B02284FF00300F4D920E7E1
:102B7000306A20F001003062306A20F004003062D8
:102B8000FFF7E8FB054641F2883700BF306A80074F
:102B900020D5FFF7DFFB401BB8424FF00300F5D90B
:102BA00007E700BF306A40F004003062306A40F04E
:102BB00001003062FFF7CEFB054641F2883700BFC7
:102BC000306A800706D4FFF7C5FB401BB842F7D92F
:102BD00037E000BFB8F1000F7FF4D5AEF06920F008
:102BE0008050F061CFE600BF306820F48030306064
:102BF000306820F480203060FFF7ACFB054600BF52
:102C0000306880037FF59DAEFFF7A4FB401B64286E
:102C10004FF00300F4D9CCE6306840F480203060F7
:102C2000306840F480303060FFF794FB054600BF09
:102C3000306880033FF585AEFFF78CFB401B6428AE
:102C4000F6D9032002B0BDE8F08100BF206AB0F5DC
:102C5000803F05D17168A26821F400311143716091
:102C60007168626A21F47411114308437060012095
:102C70003866FFF76FFB0446306880013FF598AE79
:102C8000FFF768FB001B02284FF00300F4D990E621
:102C900070B538B10446406A30B10020206104F1BB
:102CA000140007E0012070BD6068B0F5827F03D09A
:102CB00004F11C00002101600026A66294F8510076
:102CC00020B9204684F8506000F038F8022084F8DB
:102CD000510094E8071001F48271036802F4044281
:102CE00023F040030360236911440CF40062114493
:102CF00003F002026369114403F00102A369E5696C
:102D0000114403F40072114405F03802256A11449D
:102D100005F08002A56A114305F4005211430160D9
:102D2000042101EA13414160C16921F40061C161DC
:102D30000120666584F85100304670BD80B586B0CC
:102D400043F600010068C4F20001002288420492A8
:102D500002D006B080BD00BF41F21800C4F20200EC
:102D6000426842F480424260426802F4804201922A
:102D7000019A026842F008020260006800F0080050
:102D8000019001984FF4204002900220039003200C
:102D9000059001F5544002A9FFF7C8F906B080BDBF
:102DA0002DE9F04182B0044690F85000012803D18B
:102DB000022002B0BDE8F08101201D4616460F46F4
:102DC00084F85000FFF7C6FA94F8511001290DD18C
:102DD0008046002F4FF0010018BF002E0ED10021B9
:102DE00084F8501002B0BDE8F08100BF022000213D
:102DF00084F8501002B0BDE8F08100BF032000212C
:102E000084F8510061652763A686E686A163A187E1
:102E1000E187A0682164B0F5004F2068616407D1A4
:102E2000016821F040010160016841F480410160C6
:102E30000168490603D4016841F0400101606168FE
:102E4000731EE268B1FA81F1B3FA83F349095B09B1
:102E5000B2F5006F41EA03013CD131B137F8021BF2
:102E6000C1602763E08E0138E086E08E00286BD0D9
:102E7000681C0CD11DE000BF216B31F8022BC26031
:102E80002163E08E0138E086E08E00285CD0206867
:102E900081688907F0D4FFF75DFAA0EB0800A8422B
:102EA000F2D3032071E000BFFFF754FAE08E002850
:102EB0004AD0206881688907F6D5216B31F8022B4A
:102EC000C2602163E08E0138E086E08E0028F0D1F8
:102ED0003AE000BF39B139780173206B01302063CB
:102EE000E08E0138E086E08E70B3681C0BD11BE0E9
:102EF000216B09780173206B01302063E08E01386B
:102F0000E086E08E00B3206881688907F0D4FFF77F
:102F100021FAA0EB0800A842F3D3032035E000BF5C
:102F2000FFF718FAE08E78B1206881688907F7D535
:102F3000216B09780173206B01302063E08E01382A
:102F4000E086E08E0028EFD1204680212A464346C5
:102F500000F08CFC28B1606D40F0200060652020FE
:102F60006065A06838B9002001902068C1680191AF
:102F7000806801900198606D30B10120002184F8D3
:102F8000501002B0BDE8F0810020012184F85110FA
:102F9000002184F8501002B0BDE8F081411E0020ED
:102FA000B0EB116F1CBF012070474EF21002CEF241
:102FB000000251604EF62351CEF20001F0230B7057
:102FC0000721906011607047704700007047000053
:102FD000B0B582B0044600680168C368426901F078
:102FE0002F05202D03F0200506D12DB1204602B07B
:102FF000BDE8B04000F0B8BC5FEA017C1EBF02F043
:10300000010E03F4907212EB0E0253D1226B012ACF
:1030100005D111F0100218BF13F0100236D10A06C4
:1030200022D513F080021FD094F8411021293FD1FE
:10303000A168B1F5805F03D12169002900F0708299
:10304000216A4A1C226209784160E18C01390A0434
:10305000E1842DD1C16821F08001C160C16841F0D7
:103060004001C16002B0B0BD490621D513F0400156
:103070001ED0C16821F04001C1602021204684F8A3
:10308000411002B0BDE8B04000F00CBB002101913E
:10309000016801914168019101994069400613D48A
:1030A000A08DE18DE28D002A18BF884240F0BA81E0
:1030B00002B0B0BDCA0718BF13F4807240F0B680EA
:1030C0004A0700F1B980BEE0E06B016849688AB246
:1030D000002AEDD0A38D9A42EAD2E18580692028AA
:1030E00000F09C80206850E8030F216820F4807075
:1030F00041E80302DAB1206850E8030F216820F4A8
:10310000807041E8030292B1206850E8030F216803
:1031100020F4807041E803024AB1206850E8030FB0
:10312000216820F4807041E80302002ADAD1206887
:1031300050E8050F216820F0010041E80502DAB1EE
:10314000206850E8050F216820F0010041E80502E1
:1031500092B1206850E8050F216820F0010041E895
:1031600005024AB1206850E8050F216820F00100EF
:1031700041E80502002ADAD1206850E8050F2168ED
:1031800020F0400041E80502DAB1206850E8050F60
:10319000216820F0400041E8050292B1206850E823
:1031A000050F216820F0400041E805024AB120687F
:1031B00050E8050F216820F0400041E80502002A90
:1031C000DAD1202084F8420000202063206850E8F3
:1031D000030F216820F0100041E80302DAB12068F3
:1031E00050E8030F216820F0100041E8030292B17B
:1031F000206850E8030F216820F0100041E8030226
:103200004AB1206850E8030F216820F0100041E81F
:103210000302002ADAD1E06BFEF7F6FE02206063BB
:10322000A08DE18D401A81B2204674E1626C42F0BB
:10323000010262644A0706D5BEF1000F03D0626C3A
:1032400042F0020262648A0706D5BEF1000F03D085
:10325000626C42F004026264BCF1000F09D545EAD9
:103260000E02B2FA82F2520903D1626C42F00802F5
:103270006264626C002A3FF41BAF11F0200118BF9A
:10328000002D03D0204600F06FFB20684069616C80
:1032900000F0400001F00801401800F0B58000BFC8
:1032A000206850E8030F216820F4907041E8030281
:1032B000BAB3206850E8030F216820F4907041E809
:1032C000030272B3206850E8030F216820F4907065
:1032D00041E803022AB3206850E8030F216820F474
:1032E000907041E80302002ADAD11AE0206850E821
:1032F000050F216820F0010041E80502DAB12068DD
:1033000050E8050F216820F0010041E8050292B164
:10331000206850E8050F216820F0010041E805020F
:103320004AB1206850E8050F216820F0010041E80B
:103330000502002ADAD1206B012824D1206850E848
:10334000030F216820F0100041E80302DAB1206881
:1033500050E8030F216820F0100041E8030292B109
:10336000206850E8030F216820F0100041E80302B4
:103370004AB1206850E8030F216820F0100041E8AE
:103380000302002ADAD1202084F8420000202063C2
:103390002068406940063FD5206850E8050F216845
:1033A00020F0400041E80502DAB1206850E8050F3E
:1033B000216820F0400041E8050292B1206850E801
:1033C000050F216820F0400041E805024AB120685D
:1033D00050E8050F216820F0400041E80502002A6E
:1033E000DAD1E06BC0B143F65D11C0F60001416374
:1033F000FEF72EFE00283FF45BAEE06B416B02B09F
:10340000BDE8B040084700BF2046FFF7DFFD0020C1
:10341000606402B0B0BD00BF204602B0BDE8B0405D
:10342000FFF7D4BD401A216851E8031F226821F438
:10343000907142E80313DBB1216851E8031F226851
:1034400021F4907142E8031393B1216851E8031FFE
:10345000226821F4907142E803134BB1216851E8CE
:10346000031F226821F4907142E80313002BDAD184
:10347000216851E8051F226821F0010142E8051387
:10348000DBB1216851E8051F226821F0010142E803
:10349000051393B1216851E8051F226821F001014D
:1034A00042E805134BB1216851E8051F226821F05D
:1034B000010142E80513002BDAD1202184F84210E3
:1034C00000212163216851E8031F226821F01001C7
:1034D00042E80313DBB1216851E8031F226821F0A1
:1034E000100142E8031393B1216851E8031F2268D9
:1034F00021F0100142E803134BB1216851E8031F8A
:10350000226821F0100142E80313002BDAD10222D5
:1035100081B22046626302B0BDE8B040FFF754BDFF
:10352000216A31F8022B6FF35F22426021628CE541
:10353000002804BF0120704710B5044690F84100F0
:1035400028B9002084F84000204600F063F82420C9
:1035500084F841002068D4E90212C36823F40053C0
:10356000C360036923F440531A430261D4E904237E
:103570001143C268194341F20C639A431143C1607D
:103580004169A26921F44071114343F60002C4F27B
:1035900001029042416103D0FFF778F902E000BFD9
:1035A000FFF788F96268192148439100B0FBF1F0F8
:1035B00048F21F51C5F2EB11A0FB01235A094FF647
:1035C0009C73C0F6FF7302FB0300322303EB001071
:1035D000A0FB0101F02303EA5113206803EB021260
:1035E000C1F3431111448160016921F490410161EB
:1035F000416921F02A014161C16841F40051C16073
:1036000000202021606484F8411084F84210606337
:1036100010BD000070B586B040F60004C4F201048D
:10362000006804F5405100268842049602D006B096
:1036300070BD00BF41F21800C4F20200016802AD83
:1036400041F480410160016801F4804101910199D8
:10365000016841F0040101600068294600F004009F
:10366000019001984FF40070029002200390032013
:1036700005902046FEF75AFD4FF48060CDE9020622
:10368000204629460496FEF751FD25200021002200
:10369000FEF7E2FE2520FEF7CBFE06B070BD00006F
:1036A0007047000070470000FEE7000010B584B0CE
:1036B00040F2104042F20041C2F20000C4F20101A7
:1036C0004FF4807C012400234FF4602280E80A102C
:1036D000022104730375C2610161FEF71DFA00281F
:1036E00018BFFEF749F90920CDE90104072003902E
:1036F00040F21040C2F2000001A9FEF743F9002891
:1037000018BFFEF739F9082001900220029040F21C
:103710001040C2F2000001A9FEF734F9002818BFDA
:10372000FEF72AF904B010BD2DE9F04784B041F24C
:103730001800C4F20200016840F6004A41F010018E
:1037400001600168C4F2010A01F0100100910099C2
:1037500001680AF5806541F02001016001680022DE
:1037600001F020010091009901684FF4804641F07A
:103770000801016001684FF0000901F008010091A3
:103780000099016841F00401016000684FF4804134
:1037900000F00400009000982846FEF7D5FD504642
:1037A0004FF4A04100224FF4A048FEF7CDFD009653
:1037B0006E460127022428463146CDE9017903945B
:1037C000FEF7B4FC50463146CDE90087CDE90294BE
:1037D000FEF7ACFC04B0BDE8F087000080B540F215
:1037E000404043F60001C2F20000C4F200014FF471
:1037F000827200234FF4007C80E80E000A21C0E9A9
:103800000333C0E9053CC361C0E90833C0E90A31AC
:10381000FFF73EFA002808BF80BDBDE88040FEF7F4
:10382000ABB8000080B540F2984043F60001C2F208
:103830000000C4F2010100234FF00C0C4FF4E13200
:1038400080E80E00C0E90333C0E905C3C361FFF798
:103850006FFE002808BF80BDBDE88040FEF78CB831
:10386000FEE70000FEE70000704700002DE9F04190
:1038700082B01E4690460D460446FEF76BFD301A98
:1038800000EB0807FEF766FD40F20801C2F20001F6
:103890000968C1F3CB317943019121688A682A40D4
:1038A000AA4227D1064618F101001FD0FEF752FDAB
:1038B000801BB84222D2019801990028A1F1010190
:1038C00001912168896808BF074601EA0500A842FE
:1038D000ECD00FE088682840A8420BD188682840C7
:1038E000A84207D188682840A84203D188682840A8
:1038F000A842EFD0002002B0BDE8F081D4E9000179
:103900004268B1F5827F22F0E00242600AD1A168EC
:10391000B1F5004F02D0B1F5806F03D1016821F0FD
:1039200040010160A16AB1F5005F07D1016821F48F
:1039300000510160016841F400510160012084F8E8
:103940005100002084F85000032002B0BDE8F0814F
:1039500070470000FEF704BD70470000406A002178
:10396000C185C184FFF732BB81B090F84210222993
:1039700021D183680246B3F5805F09D152F8281F30
:1039800052F8183C002B63D003685B680AE000BF64
:1039900052F8281F13B90369002BF5D003685B6840
:1039A00003F07F030B70116801311160C18D013983
:1039B0000A04C18502D001B0704700BF0168CA681F
:1039C00022F02002CA60CA6822F48072CA604A6982
:1039D00022F001024A61202180F842100021416357
:1039E000026B012A3CD10163016851E8031F0268A0
:1039F00021F0100142E80313DBB1016851E8031F15
:103A0000026821F0100142E8031393B1016851E804
:103A1000031F026821F0100142E803134BB1016853
:103A200051E8031F026821F0100142E80313002B44
:103A3000DAD101680A68D20606D5002200920A6827
:103A40000092496800910099818D01B0FFF7BCBADE
:103A5000026852686FF35F2221F8022B8162A5E7AA
:103A600001B0FFF71DBE000040F29840C2F2000016
:103A7000FFF7AEBAFEE7000096B0FEF77FFC002429
:103A80000120CDE91144CDE90F440C9010904FF482
:103A9000E0104FF48031022515900CA80694CDE972
:103AA0000444CDE90D14CDE91351FEF717FF28B1F9
:103AB000EFF3108072B600BFFEE700BF0F20CDE924
:103AC00007054FF48060CDE90A0407A80221099494
:103AD000FEF7FCFD20B1EFF3108072B6FEE700BFE9
:103AE000022003904FF40040059003A8FEF768FD04
:103AF00020B1EFF3108072B6FEE700BFFFF714FEAF
:103B0000FFF7D4FDFFF78EFEFFF768FE0CA8FDF768
:103B1000FFFE40F21047C2F200073846FEF70EFAE9
:103B200038460A21FEF7D6F8012508264FF4FA7028
:103B3000FEF7E8FA3846FDF7EBFF0D9C82B2002055
:103B40000021042300960195A0470D9C0020092127
:103B50000022042300960195A04714988047384618
:103B6000FDF7D6FF0D9C82B20020002104230096B1
:103B70000195A0470D9C00200921002204230096F6
:103B80000195A04714988047D0E702E008C8121FAB
:103B900008C1002AFAD170477047002001E001C136
:103BA000121F002AFBD17047000000000000000037
:103BB00001020304060708090000000001020304D3
:103BC00001020000F010101010FF10101010F00093
:103BD000000000000F04040404FF040404040F00A8
:103BE00000004040405F555555755555555F404064
:103BF00040000040200F094989790909090F204038
:103C0000000000FE02424ACA4A4ACA4A4A4202FE2A
:103C1000000000FF40504C4340404F50505C40FF7C
:103C200000000000F888888888FF88888888F80065
:103C3000000000001F080808087F888888889F8087
:103C4000F00080828282828282E2A2928A868280D0
:103C50008000000000000040807F000000000000A5
:103C60000000101010FF109008888888FF8888884E
:103C700008000444827F01808040432C1028468144
:103C800080000010101010D030FF30D0121C101027
:103C9000000010080402010000FF000001020408F7
:103CA000100004040484E43C2724242424E40404B1
:103CB000040004020100FF0909090949897F000085
:103CC000000000FE225A8600FE9292929292FE001E
:103CD000000000FF04080700FF4020030C142241ED
:103CE0004000008040201806800007182040800017
:103CF00000000100207028262120202438600001C7
:103D00000100001012929292929292121202FE0000
:103D100000000000003F101010103F0040807F00A6
:103D20000000000000C080808080808080FC848053
:103D30008080808080C0C0000000000000FF7F40C5
:103D40004040404040FF40404040404040FF7F00F6
:103D5000000000000000000000000000007F700074
:103D60000000000000000000000000000000000053
:103D7000000000000000000000FCF800000000004F
:103D80000000000000000000000000000000FFFE36
:103D9000020202020202020202FFFF020202020209
:103DA00002020202FF0300000000000000001F1FCB
:103DB000040404040404040404FFFF0404040404CD
:103DC000040404041F0000000000000000000000C4
:103DD0000000000000000000007F3F000000000025
:103DE00000000000000000000000000000000000D3
:103DF00000000000000000000000000000000000C3
:103E000000000000000000F8F8F0F0702000000052
:103E100000000000000000000000000000000000A2
:103E20000000000000000000000000000000000092
:103E30000000800000000000000000000000000002
:103E400000000000000000FFFFFFFF000000000076
:103E50000000000000000000000000000000808062
:103E60000000000000000000000000000000000052
:103E7000000000FFFFFE060606060606060606060A
:103E800006060606060606FFFFFFFF0606060606EE
:103E900006060606060606060606060606FFFFFFD7
:103EA000FF0702000000000000000000000000000A
:103EB000000000FFFFFF0000000000000000000005
:103EC00000000000000000FFFFFFFF0000000000F6
:103ED00000000000000000000000000000FFFFFFE5
:103EE000FF000000000000000000000000000000D3
:103EF000000000FFFFFF18181818181818181818D5
:103F000018181818181818FFFFFFFF181818181895
:103F100018181818181818181818181818FFFFFF6C
:103F2000FF00000000000000000000000000000092
:103F3000000002010100000000000000000000007D
:103F400000000000000000FFFFFFFF000000000075
:103F5000000000000000000000000000000101005F
:103F60000000000000000000000000000000000051
:103F70000000000000000000000000000000000041
:103F800000000000000000FFFFFFFF000000000035
:103F90000000000000000000000000000000000021
:103FA0000000000000000000000000000000000011
:103FB0000000000000000000000000000000000001
:103FC000000000000000001F1F0F0F000000000095
:103FD00000000000000000000000000000000000E1
:103FE00000000000000000000000000000000000D1
:103FF0000000002F000000000700070000147F14DD
:104000007F1400242A7F2A120062640813230036DA
:104010004955225000000503000000001C22410009
:10402000000041221C000014083E08140008083E4D
:104030000808000000A06000000808080808000048
:1040400060600000002010080402003E5149453E17
:104050000000427F40000042615149460021414535
:104060004B31001814127F10002745454539003C9C
:104070004A4949300001710905030036494949366A
:1040800000064949291E0000363600000000563659
:10409000000000081422410000141414141400003D
:1040A0004122140800020151090600324959513ECB
:1040B000007C1211127C007F49494936003E414183
:1040C0004122007F4141221C007F49494941007F34
:1040D00009090901003E4149497A007F0808087F23
:1040E0000000417F4100002040413F01007F081453
:1040F0002241007F40404040007F020C027F007F51
:104100000408107F003E4141413E007F0909090635
:10411000003E4151215E007F091929460046494968
:1041200049310001017F0101003F4040403F001F35
:104130002040201F003F4038403F006314081463B4
:1041400000070870080700615149454300007F419E
:10415000410000552A552A55000041417F000004C6
:1041600002010204004040404040000001020400FF
:10417000002054545478007F484444380038444464
:10418000442000384444487F0038545454180008F0
:104190007E0901020018A4A4A47C007F080404780E
:1041A0000000447D4000004080847D00007F102896
:1041B00044000000417F4000007C04180478007C2B
:1041C0000804047800384444443800FC24242418AB
:1041D0000018242418FC007C0804040800485454E7
:1041E000542000043F444020003C4040207C001C00
:1041F0002040201C003C4030403C00442810284413
:10420000001CA0A0A07C004464544C44141414145A
:104210001414000000000000000000000000000076
:10422000FC000000000002000000000C020C020074
:1042300000000000000090D0BCD0BC900003000340
:1042400000001824FE448C00030207020100182419
:10425000D8B04C80000300010201C038E438E0000F
:104260000102020102020806000000000000000036
:104270000000000000F80402000000010204000237
:1042800004F800000004020100009060F860900053
:104290000000010000002020FC20200000000100A0
:1042A00000000000000000000806000000002020C0
:1042B000202020000000000000000000000000009E
:1042C0000002000000000080601C020004030000E7
:1042D0000000F8040404F8000102020201000008D2
:1042E000FC000000000203020000188444241800AF
:1042F00003020202020008042424D8000102020280
:10430000010040B088FC80000000000302003C2453
:104310002424C400010202020100F824242CC0005D
:104320000102020201000C04E41C0400000003006E
:104330000000D8242424D8000102020201003844DD
:104340004444F800000302020100000010000000D5
:104350000000020000000000200000000000060035
:10436000000000205088040200000000010290902C
:10437000909090000000000000000002048850208F
:104380000002010000001804C4241800000002000C
:104390000000F804E494F80001020202020000E0C8
:1043A0009CF0800002030000030204FC2424D800D7
:1043B000020302020100F80404040C0001020202DC
:1043C000010004FC0404F80002030202010004FCE2
:1043D00024740C0002030202030004FC24740C0089
:1043E000020302000000F0080444CC400001020275
:1043F000010004FC2020FC0402030000030204046A
:10440000FC040400020203020200000404FC040491
:1044100006040403000004FC24D00C040203020080
:10442000030204FC04000000020302020203FC3C3D
:10443000C03CFC0003000300030004FC30C4FC0487
:10444000020302000300F8040404F800010202025F
:10445000010004FC24241800020302000000F88478
:104460008404F80001020207050004FC246498009B
:10447000020302000302182424448C0003020202F7
:1044800001000C04FC040C0000020302000004FC08
:104490000000FC04000102020100047C80E01C0416
:1044A0000000030000001CE03CE01C0000030003CF
:1044B0000000049C609C0400020300030200041C32
:1044C000E01C04000002030200000C84641C0400D1
:1044D0000203020203000000FE02020000000704C3
:1044E0000400000E30C000000000000102000002C5
:1044F00002FE0000000404070000000402040000A3
:10450000000000000000000000000000080808088B
:104510000808000002000000000000000000004049
:10452000A0A0C00000010202030204FC2020C00081
:1045300000030202010000C020206000000102020E
:10454000020000C02024FC0000010202030200C09F
:10455000A0A0C0000001020202000020F8242404F0
:104560000002030202000040A0A0602000070A0A27
:104570000A0404FC2020C000020302000302002001
:10458000E4000000000203020000000020E400003C
:1045900008080807000004FC80E020200203020055
:1045A00003020404FC000000020203020200E020F7
:1045B000E020C00003000300030020E02020C00032
:1045C00002030200030200C02020C000000102021A
:1045D000010020E02020C000080F0A02010000C0F6
:1045E0002020E0000001020A0F0820E04020200007
:1045F0000203020000000060A0A0200000020202EE
:1046000003000020F820000000000102020020E06A
:104610000020E00000010202030220E02080602070
:104620000000030100006080E080600000030003E0
:10463000000020608060200002030003020020E0F0
:10464000208060200808070100000020A0602000F2
:10465000000203020200000020DE0200000000074A
:104660000400000000FF00000000000F0000000236
:10467000DE20000000040700000002010204040222
:10468000000000000000000000000000000000002A
:10469000000000000000000000F800000000000022
:1046A00000333000000000100C06100C0600000063
:1046B00000000000000040C07840C0784000043F87
:1046C00004043F040400007088FC08300000001857
:1046D00020FF211E0000F008F000E018000000217B
:1046E0001C031E211E0000F00888700000001E211F
:1046F00023241927211010160E00000000000000CE
:10470000000000000000000000E0180402000000AB
:1047100000071820400000020418E00000000040DC
:10472000201807000000404080F080404000020256
:10473000010F01020200000000F000000000010172
:10474000011F01010100000000000000000080B016
:1047500070000000000000000000000000000001E8
:104760000101010101010000000000000000003013
:1047700030000000000000000000806018040060AD
:1047800018060100000000E010080810E000000F0B
:10479000102020100F00001010F800000000002072
:1047A000203F2020000000700808088870000030BA
:1047B0002824222130000030088888483000001862
:1047C000202020110E000000C02010F8000000077B
:1047D0000424243F240000F80888880808000019F1
:1047E000212020110E0000E0108888180000000F22
:1047F000112020110E0000380808C83808000000F9
:10480000003F000000000070880808887000001C4D
:10481000222121221C0000E010080810E000000006
:10482000312222110F00000000C0C0000000000073
:104830000030300000000000008000000000000098
:10484000806000000000000080402010080000018F
:104850000204081020004040404040404000040452
:10486000040404040400000810204080000000201C
:10487000100804020100007048080808F000000059
:10488000003036010000C030C828E810E0000718EA
:10489000272423140B000000C038E0000000203C57
:1048A00023020227382008F8888888700000203FFB
:1048B000202020110E00C030080808083800071812
:1048C00020202010080008F808080810E000203F09
:1048D000202020100F0008F88888E8081000203FEA
:1048E00020202320180008F88888E8081000203FBE
:1048F000200003000000C030080808380000071836
:104900002020221E020008F808000008F808203FB6
:10491000210101213F20000808F8080800000020BC
:10492000203F2020000000000808F8080800C08090
:1049300080807F00000008F888C028180800203F09
:1049400020012638200008F8080000000000203F61
:1049500020202020300008F8F800F8F80800203F58
:10496000003F003F200008F830C00008F808203F52
:10497000200007183F00E01008080810E0000F10A2
:10498000202020100F0008F808080808F000203F39
:10499000210101010000E01008080810E0000F18D4
:1049A000242438504F0008F8888888887000203FF9
:1049B0002000030C302000708808080838000038F8
:1049C000202121221C00180808F8080818000000FF
:1049D000203F2000000008F808000008F808001F29
:1049E000202020201F000878880000C83808000018
:1049F00007380E010000F80800F80008F800033C32
:104A00000700073C030008186880806818082030F9
:104A10002C03032C30200838C800C83808000000D8
:104A2000203F2000000010080808C838080020387F
:104A3000262120201800000000FE020202000000D3
:104A4000007F40404000000C30C00000000000002B
:104A500000010638C00000020202FE000000004013
:104A600040407F0000000000040202020400000039
:104A70000000000000000000000000000000808036
:104A8000808080808080000202040000000000001E
:104A900000000000000000008080808000000019FD
:104AA000242222223F2008F8008080000000003FDE
:104AB000112020110E000000008080800000000EF8
:104AC000112020201100000000808088F800000ED6
:104AD000112020103F200000808080800000001FF7
:104AE000222222221300008080F08888881800206B
:104AF000203F202000000000808080808000006B2C
:104B000094949493600008F8008080800000203F17
:104B1000210000203F200080989800000000002025
:104B2000203F20200000000000809898000000C076
:104B30008080807F000008F8000080808000203F97
:104B400024022D302000000808F80000000000209A
:104B5000203F202000008080808080808000203FD7
:104B600020003F20003F8080008080800000203FA8
:104B7000210000203F200000808080800000001F76
:104B8000202020201F00808000808000000080FF07
:104B9000A12020110E000000008080808000000E07
:104BA000112020A0FF808080800080808000202055
:104BB0003F212000010000008080808080000033C1
:104BC000242424241900008080E08080000000005C
:104BD000001F202000008080000000808000001F57
:104BE000202020103F2080808000008080800001F5
:104BF0000E300806010080800080008080800F3029
:104C00000C030C300F0000808000808080000020AA
:104C1000312E0E31200080808000008080808081D5
:104C20008E70180601000080808080808000002146
:104C3000302C2221300000000000807C02020000A5
:104C40000000003F404000000000FF0000000000A6
:104C50000000FF0000000002027C80000000004015
:104C6000403F0000000000060101020204040000B1
:104C70000000000000000000000000000000000034
:104C80000000000000000000000000000000000024
:104C9000000000000000000000000000000000F024
:104CA000F0F0000000000000000000017F010000A3
:104CB000000000000000001C1C1C000000000000A0
:104CC0008060301C8C60301C0C0000000000000074
:104CD00000000000000000000000000000000000D4
:104CE0000000000000E00000000000E0000000867E
:104CF000E69F86868686E69F860000011F010101E9
:104D000001011F010100000080C06020F820E0C008
:104D10000000000003070C18FF70E1810000000094
:104D2000070F10107F100F070000806020608000C8
:104D30000000E02000000F3020309F70DC37103082
:104D4000C0000000100E0300071810180700000034
:104D5000C02020E0C0000000000080E01F38E8878D
:104D600003C43C040000070F1810100B070D1010AF
:104D7000080000808C4C380000000000000000009B
:104D80000000000000000000000000000000000023
:104D900000000000000000000000000080E030087B
:104DA00004000000000000FEFF0100000000000001
:104DB00000000000030F1820400000040830E080CD
:104DC0000000000000000000000001FFFE000000E5
:104DD0000000004020180F03000000000000000049
:104DE00000000000C00000000000004266663C18A1
:104DF000FF183C666642000000000000030000004F
:104E00000000000000000000800000000000001012
:104E100010101010FF101010101000000000000003
:104E2000030000000000000000000000000000007F
:104E300000000000000000000000000000000080F2
:104E40008C4C380000000000000000000000000052
:104E500000000000000000101010101010101010C2
:104E60001000000000000000000000000000000032
:104E70000000000000000000000000000000000032
:104E800000000000000000001C1C1C0000000000CE
:104E900000000000000000000000E0380C000000EE
:104EA000000080701C03000000000060380E01004C
:104EB000000000000000000080C060202060C08072
:104EC000000000FEFF010000000001FFFE000001E5
:104ED000070E181010180E0701000000808080C017
:104EE000E000000000000000000000FFFF000000E4
:104EF000000000001010101F1F1010100000008094
:104F0000402020202060C08000000003030080407B
:104F100020381F070000001C1A1918181818181F2D
:104F200000000080C020202060C08000000000033E
:104F300003001010182FE780000000070F1010105A
:104F400010180F070000000000000000C0E0F00093
:104F5000000000C0B088868180FFFF8080000000D4
:104F600000000010101F1F1010000000E0606060C3
:104F700060606060000000003F1008080818F0E062
:104F8000000000070B101010101C0F0300000000A1
:104F900080C040202020E0C0000000FCFF2110085D
:104FA000080818F0E0000001070C18101010080F96
:104FB00003000000C0E06060606060E0600000002E
:104FC00003000000E0180700000000000000001FC0
:104FD0001F00000000000080C0602020202060C072
:104FE00080000087EF2C1818303068CF830000074E
:104FF0000F0810101010180F07000000C0C020206C
:105000002020C0800000001F3F604040402010FF73
:10501000FE0000000C1C101010080F030000000020
:105020000000000000000000000000000000000E72
:105030000E0E0000000000000000001C1C1C000000
:105040000000000000000000000000000000000060
:105050000000000C0C0000000000000000000058E0
:105060003800000000000000000000000080402028
:105070001000000010284482010000000000000021
:105080000000000001020408100000000000000001
:10509000000000000000008484848484848484846C
:1050A000840000000000000000000000000000007C
:1050B0001020408000000000000000000000000000
:1050C00001824428100000001008040201000000C2
:1050D000000000C020201010101030E0C0000003BD
:1050E000030000F010080C070300000000001C1C67
:1050F0001C0000000000000000C040602020204094
:10510000C00000FCFF01F00E03C1FE03807F000120
:10511000070E08111110110904020000000080E0C0
:10512000E000000000000000807C4340477FF880E2
:10513000000010181F1000000000131F1C1020E0BA
:10514000E02020202060C080000000FFFF10101031
:1051500010182FE78000101F1F1010101010180FCC
:105160000700000080C0402020202060E00000FCFC
:10517000FF0100000000000001000001070E1810F0
:1051800010100804030020E0E02020202040C08010
:10519000000000FFFF000000000001FFFE00101FE4
:1051A0001F10101018080E07010020E0E02020203A
:1051B00020202060800000FFFF101010107C0000F5
:1051C0000000101F1F10101010101018060020E013
:1051D000E020202020206060800000FFFF101010E1
:1051E000107C00000100101F1F10000000000000D4
:1051F0000000000080C06020202040E0000000FC93
:10520000FF0100004040C0C140400001070E1810DF
:1052100010100F0F000020E0E0200000000020E050
:10522000E02000FFFF101010101010FFFF00101FF3
:105230001F1000000000101F1F100000202020E0A1
:10524000E020202000000000000000FFFF00000020
:10525000000000001010101F1F10101000000000B0
:105260000000202020E0E0202020000000000000BE
:1052700000FFFF0000000060E0808080C07F3F00F2
:10528000000020E0E020000020A06020200000FFBF
:10529000FF30187CE3C000000000101F1F1000004A
:1052A00001131F1C181020E0E02000000000000087
:1052B000000000FFFF000000000000000000101FC1
:1052C0001F10101010101018060020E0E0E0000081
:1052D0000000E0E0E02000FF013FFEC0E01E01FF13
:1052E000FF00101F1000031F0300101F1F1020E0FD
:1052F000E0C0000000000020E02000FF0003071CC9
:1053000078E08000FF00101F100000000000030F75
:105310001F00000080C060202060C080000000FEF0
:10532000FF010000000000FFFE000001070E181042
:1053300010180C07010020E0E0202020202060C091
:10534000800000FFFF2020202020301F0F00101FB2
:105350001F100000000000000000000080C060205E
:105360002060C080000000FEFF010000000000FF80
:10537000FE000001070E1111133C7C67210020E0A4
:10538000E0202020202060C0800000FFFF101030AF
:10539000F0D0080F0700101F1F10000000030F1CA3
:1053A00010100080C060202020204040E000000756
:1053B0000F0C1818303060E08100001F0C0810102E
:1053C0001010180F07008060202020E0E02020202F
:1053D00060800100000000FFFF00000000010000ED
:1053E0000000101F1F100000000020E0E02000005F
:1053F00000000020E02000FFFF000000000000008F
:10540000FF0000070F181010101010080700206090
:10541000E0E02000000020E060200000077FF8802E
:1054200000807C03000000000000071F1C07000034
:10543000000020E0E02000E0E0200020E020000765
:10544000FFF8E01FFFFCE01F00000000031F030047
:10545000011F03000000002060E0A0000020E060C9
:105460002000000000038F7CF8C60100000000103F
:10547000181E130001171F1810002060E0E0200024
:10548000000020E06020000001073EF8E01807005F
:10549000000000000010101F1F101000000000800E
:1054A0006020202020A0E0E0200000000000C0F0EC
:1054B0003E0F0300000000101C1F171010101018E2
:1054C00006000000000000FC0404040404000000C6
:1054D000000000FF00000000000000000000007F4E
:1054E000404040404000000010E00000000000008C
:1054F000000000000000031C6080000000000000AD
:105500000000000000030C7080000000040404048C
:1055100004FC0000000000000000000000FF00008C
:105520000000000040404040407F000000000000BC
:105530000010080C040C081000000000000000001F
:10554000000000000000000000000000000000005B
:10555000000000000000000000000000000000004B
:10556000000000000000000000008080808080803B
:105570008080808080800000000404080800000013
:10558000000000000000000000000000000000001B
:10559000000000000000000000000000000000000B
:1055A000000000000000000098D844642424FCF8A7
:1055B0000000000F1F18101010081F1F10180020E7
:1055C000E0F000000000000000000000FFFF1808ED
:1055D00004040CF8F00000001F0F18101010180F32
:1055E000030000000000000000000000000000E0D8
:1055F000F8180404043C3800000000030F0C1010DD
:105600001010080600000000000000000020E0F07C
:10561000000000E0F81C04040408FFFF0000000381
:105620000F18101010081F0F0800000000000000E5
:105630000000000000000000E0F8484444444C78BA
:1056400070000000030F0C18101010080400000078
:10565000000080C0602020E0C00000040404FFFFC0
:10566000040404040000000010101F1F101010009C
:10567000000000000000000000000000000000002A
:1056800070F88C04048CF874040C007076CF8D8D47
:105690008D89C87870000020E0F000000000000054
:1056A00000000000FFFF08040404FCF800000010E4
:1056B0001F1F100000101F1F1000000000000060DE
:1056C0006000000000000000040404FCFC00000076
:1056D000000000001010101F1F101010000000002C
:1056E00000000000006060000000000000000404F2
:1056F00004FCFC0000000000C0C08080C07F3F00B0
:1057000000000020E0F000000000000000000000A9
:10571000FFFF80C0F41C0404000000101F1F1100D4
:10572000031F1C1010000000202020E0F0000000EB
:1057300000000000000000FFFF000000000000006B
:105740001010101F1F1010100000000000000000BB
:1057500000000000000004FCFC0804FCFC0804FC41
:10576000FC00101F1F10001F1F10001F1F10000043
:10577000000000000000000000000004FCFC08081D
:105780000404FCF8000000101F1F100000101F1F71
:10579000100000000000000000000000000000E019
:1057A000F0180C04040C18F0E00000030F0C1010AB
:1057B00010100C0F030000000000000000000000AB
:1057C00000000004FCFC080404040CF8F000008055
:1057D000FFFF889010101C0F030000000000000065
:1057E00000000000000000E0F81C04040408F8FCBD
:1057F000000000030F1810109088FFFF80000000C9
:1058000000000000000000000000040404FCFC1084
:105810000804040C0C001010101F1F1010100000C2
:105820000000000000000000000000000000000078
:105830003078CCC48484840C1C0000001E18101026
:105840001011190F06000000000000C00000000049
:10585000000000040404FFFF040404000000000032
:1058600000000F1F1010100C0000000000000000CE
:105870000000000000000004FCFE00000004FCFE2C
:10588000000000000F1F181010081F0F0800000074
:105890000000000000000000000000040C3CFCC4FC
:1058A0000000C43C0C0400000000010F1E0E0100AB
:1058B0000000000000000000000000000000043CA8
:1058C000FCC400E47CFC84807C040000071F07000B
:1058D00000071F070000000000000000000000009B
:1058E00000000004041C7CE4C0341C04040000100C
:1058F000101C1601131F1C181000000000000000EF
:1059000000000000000000040C3CFCC400C43C0487
:1059100004000000C080C1370E010000000000003C
:105920000000000000000000000000001C0404C48F
:10593000F47C1C0400000000101C1F17111010182C
:105940000E0000000000000000F80C040000000041
:105950000000001028EF0000000000000000000020
:10596000003F60400000000000000000FF00000059
:105970000000000000000000FF0000000000000028
:1059800000000000FF00000000000000040CF80010
:1059900000000000000000000000EF2810000000E0
:1059A0000000000040603F00000000000000001800
:1059B0000602020408102020300800000000000049
:1059C00000000000000000000000000000000000D7
:1059D000000002030405060708090A0B0C0D0E0F50
:1059E00010100000085A00080000002010000000FD
:1059F0008A3B0008185A000810000020D808000050
:105A00009A3B0008000000000100000010000000A8
:085A10000024F4000000000076
:04000005080000ED02
:00000001FF
